:020000040000FA
:1000000000000D2A00340034F200030E8301F100D9
:100010000A088A01F00004088312AC008316A401C8
:1000200083120B1D15288316A40A83162408A50025
:10003000013A031D2428B030831281008316BC0AC4
:100040000319BD0A83120B118316A40183120C1F1E
:100050002B288316A40A83162408A500013A031D41
:1000600032289C2183122C088312840070088A0095
:100070008301710E8300F20E720E09008316B40123
:10008000B501B601B701B801B901703083168F040C
:10009000073083129900403083168C0083128C0144
:1000A000E0308B000B308316850083128501803091
:1000B00083168100B030831281008316BA010A30A2
:1000C00083163A02031896288312051583163C08F6
:1000D0008316B40083163D088316B500E830FD0092
:1000E0000330FE0083163408FF00350839218316DB
:1000F000BB003B0803196E288312051183163C08C8
:100100008316B40083163D088316B500E830FD0061
:100110000330FE0083163408FF00350839218316AA
:10012000BB003B0803198628BA0A5F2823308316D0
:100130009F00813083129F009F1483163E1CDE288F
:10014000831638080319A9283808013A0319C42866
:10015000EA28831285160A30FD000030FE0083165F
:100160003408FF00350839218316BA003A0803190C
:10017000EA280130B80083163C088316B4008316C1
:100180003D088316B500EA2883128512BE30FD00B3
:100190000030FE0083163408FF003508392183162D
:1001A000BA003A080319EA28B80183163C088316F6
:1001B000B40083163D088316B500EA288312851221
:1001C0008316B80183163C088316B40083163D08D5
:1001D0008316B5008316BE1C2B2983163908031914
:1001E000F6283908013A031911299D2883120516AA
:1001F0001430FD000030FE0083163608FF0037087B
:1002000039218316BA003A0803199D280130B90034
:1002100083163C088316B60083163D088316B70084
:100220009D2883120512B430FD000030FE008316B5
:100230003608FF00370839218316BA003A08031937
:100240009D28B90183163C088316B60083163D0825
:100250008316B7009D28831205128316B9018316F1
:100260003C088316B60083163D088316B7009D2808
:1002700008008316A7007F08A6007E08A9007D0855
:10028000A80083163C088316AA0083163D0883162F
:10029000AB0027082B02031D4F2926082A0203184A
:1002A000882983162608AC00AE01AF01AC090314FF
:1002B0002708AD0003185E29FE3C5F29FF3C83162A
:1002C000AD002E08031C2E0F672900306829003C62
:1002D0008316AE002F08031C2F0A003CAF002A082B
:1002E000B000B201B3012C083007AC002B08B100FC
:1002F0000318310FAD0732080318320FAE07330869
:100300000318330FAF072C08AA002D08AB008F2964
:1003100083162608AA022708031C270FAB028316A0
:1003200029082B02031D962928082A02031C9A2952
:1003300001309B2900300800033083121E0583160C
:10034000A000A300A100A201A00183161E0883162D
:10035000A100A2012108A00700300318220FA30763
:1003600003302302031DB62966302002031CD32963
:100370008316A00183121F1DBF298316A00A8316AE
:100380002008A1000319C9292108013A0319CE291F
:10039000E92983163E1483120515E9298316BE1434
:1003A00083120511E9298316A00183121F1DDA2982
:1003B0008316A00A83162008A1000319E429210846
:1003C000013A0319E729E92983163E10E929831622
:1003D000BE10003083163E04031DF1298316051557
:1003E000F329831605118316A00183121F1DFA2914
:1003F0008316A00A83162008A1000319042A2108E5
:10040000013A0319072A092A83121F15092A8312A0
:100410001F1183129F140C130800DD30FE00023000
:10042000FF00803000000000BC22000000008312AA
:100430000000A1007F08A000DF30A2000230A3006E
:10044000831200002008A4002108A500FF30A007A7
:10045000031CA103240825040319A52A043022073C
:10046000A400A501A50D2308A5072408FE00250862
:10047000FF00803000000000BC220000000083125A
:100480000000A7007F08A6002208FE002308FF0046
:10049000803000000000BC22000000008312000039
:1004A000A900A5007F08A800A40002302207A4002C
:1004B000A501A50D2308A5072408FE002508FF00B7
:1004C000803000000000BC22000000008312000009
:1004D000A500AB007F08A400AA0083120000260834
:1004E000AA002708AB00FF30A607031CA7032A08B1
:1004F0002B0403199E2A2808FE002908FF008030DB
:1005000000000000A9220000000083120000AA00E1
:100510002408831203138400831383120000251818
:1005200083172A0883120313800083120000A80A8D
:100530000319A90AA40A0319A50A6D2A0630831211
:100540000000A2070318A30A202A000000003E288A
:100550000800003A0319B02A803A0319B72A003478
:100560007E08840083137F188317000808007F0823
:100570008A007E0882000800003A0319C42A803AE3
:100580000319CE2AFF0100347E08840083137F18EC
:1005900083170008FF00840A00080800000000001C
:1005A000B722FD00FE0FFF03FF0A00000000B72284
:1005B000FC007D08FF007C08080003340034F1349F
:1005C0000234BE3400340134003402340034BC340C
:1005D000003402340034F23402342D340034013457
:0605E00000340034003479
:02400E00D430AC
:00000001FF
